:020000040000FA
:020000000528D1
:06000A00850186010730AC
:100010009F000313831686018614850183128316BD
:100020000930990018128312A301A9217F307B2186
:10003000FF007E307B21FE007D307B21FD007C3087
:100040007B21FC002F30FA006F3084007A087B217E
:1000500080008403FA0B26287A087B218000FB01AC
:100060007021A2016421B921183085009817181653
:100070008C1E4B281A08A2008D21BA17A21F8028B7
:100080002208FA00F039F03A031D5A287A08F03AAB
:1000900003192529382883168501051483120518AC
:1000A0005520831685018312382805185528061413
:1000B0007C17080022080F397C1F6E287F06031961
:1000C0006D280F302205FF0083169A007F309B00B9
:1000D000831281217C13061038287F087F06031DB8
:1000E0007E28220E0F39A200083022028207D6286D
:1000F0009C287E28FE287E287E287E28A30138287A
:100100002308FB000F307B057F06031D3828FB0EFC
:100110000F30FB057B088207382800000000000034
:100120000000000000000000DB28A1283828032977
:1001300038283828382838285F21A21B9C287A08BC
:10014000A3002208FB005F21A21BA3282208031999
:10015000E028FC1AAC2864217C1FB9287B08FE002B
:1001600083169A007E309B00831281217C13061037
:100170003828AF0A2F0884007B0880007E08FB0225
:10018000031CFB017C1AD0207C1E7B0D7021061401
:1001900039302F06031D38288030B100AF033828CE
:1001A0007B08403E84000008FB0008005F21A21B82
:1001B000D6287A08A3002208FB005F21A21BDD28B5
:1001C0002F0884007B08BA000006031D3828303051
:1001D0000406031938280403303A0319FC28840361
:1001E0000008FB007E08FB02031CFB017C1AD020E8
:1001F0007C1E7B0D70213828061038285F21A21B39
:10020000FE287A08A3002208FB005F21A21B052913
:100210007B307B06031D1129A208031D3828A92164
:10022000FC287C1F1D297B08FD0083169A007D3069
:100230009B00831281217C130610FC1E38287D0848
:100240007B06031D3828642138285F21A21B5E2904
:1002500070302206031D5E295F21A21B5E297F08E4
:100260002206031D5E2906145F21A21B5E292208B7
:10027000FA005F21A21B5E292208FB005F21A21B5E
:100280005E292208A3005F21A21F5E29230EFB071F
:100290007A0883169B007B089A00831281217A08D2
:1002A000303C031C59297A08403E84007B088000BA
:1002B0005D297A0884007B088000061038288C1E8F
:1002C0005F291A08A2000800220DF8390618013E1D
:1002D0008600220D0739083E85000000051608003B
:1002E000F8390618013E86007B0D0739103E85005F
:1002F00000008515080083169B001C141A08831241
:10030000080083161C158B1355309D00AA309D00E4
:100310009C141C118B178312080003108030AE0050
:100320003130840000083A068030031D992980008E
:10033000AF030006031DA429840A0008840380007B
:10034000840A803080008403840AAE0C031C922946
:1003500008008030B000B100B200B300B400B500B6
:10036000B600B700B800B900FF30BA003030AF00B7
:1003700008000614C5210610C5210614C521061063
:10038000C5210614C52106100800FF30FB00FF3010
:10039000FA00000000000000000000000000000063
:1003A0000000000000000000FA0BC929FB0BC72960
:0203B000080043
:02400E002A3F47
:00000001FF
